:020000040000FA
:0600000088EF07F012007A
:0600080004EF08F01200F5
:060018000CEF08F01200DD
:0E00200001003C0F0000FE0100000200000085
:02002E00F00ED2
:100030008C1695160001636B676968696969666B60
:10004000010E6A6F1200D9CFE6FFE1CFD9FFE65269
:10005000000163511FE1040108BF1BD0400EE66E92
:10006000700EE66E010EE66EB9EC05F0E552E55253
:10007000E5520001010E636FDF6A400EDF5C09E2AA
:10008000DF50EA6AB00FE96E010EEA22EF6ADF2A5A
:10009000F4D74BD101017051080A01E135D10F0AA3
:1000A00001E1F5D0010A01E1EAD0030A01E18ED0B5
:1000B000010A59E0070A4CE0010A01E036D10101CA
:1000C000020EB06F01013A0EB16F0101010EB26F65
:1000D0000101010EB36F0101B46B100EB56FB66B69
:1000E000B76B0101B86B300EB96FBA6BBB6B010116
:1000F000030EBC6F0101BD6BBE6B300EBF6FC06BDA
:1001000001010C0EC16FC26BC36BC46B0101010E08
:10011000C56F0101C66BC76B200EC86FC96B0101AB
:10012000080ECA6FCB6BCC6BCD6B0101CE6904019D
:100130000CBF0DD0400EE66EB00EE66E010EE66E00
:1001400089EC05F0E552E552E5520001636BEDD014
:100150000001010E6A6F0101715102E100016A6B39
:100160000001636BE2D0400E0001646F656B00011B
:10017000000E645D010E65591FE2040064C000F0CA
:1001800065C001F0026A060E1F0B00C0F6FF01C039
:10019000F7FF02C0F8FF06E0D890F636F736F836DB
:1001A000E806FAE1940EA66E57D91AEC06F00001A3
:1001B000642B000E6523DBD7F66AF76A200EF86E13
:1001C000940EA66E49D90001636BAFD0300E0101C9
:1001D000735D07E100016A5101E116D90001636B0B
:1001E000A4D0E8680001671905E1E868681902E130
:1001F000E868691906E171C167F072C168F073C1FE
:1002000069F0670EE96E000EEA6EEE500101711999
:1002100008E1EE500101721904E1EE500101731979
:1002200000E12AE1DF6A01017551DF5C25E23A0E47
:100230000101D8807555DF24EA6A760FE96E010E58
:10024000EA22EF50E66E00016651EA6A6B0FE96E32
:10025000000EEA22E552E750EF6E0001662B000126
:10026000672B000E6823000E6923100E0001665DE7
:1002700001E160D8DF2AD7D70001636B56D05AD886
:1002800000016769686969690001636B4ED001010B
:10029000070EB06F71C1B1F172C1B2F173C1B3F1A8
:1002A00074C1B4F175C1B5F171C1F6FF72C1F7FF48
:1002B00073C1F8FFDF6A01017551DF5C14E2F00ED3
:1002C0000101735D01E10DD009003A0E0101D880F2
:1002D0007555DF24EA6AB60FE96E010EEA22F5CF02
:1002E000EFFFDF2AE8D704010CBF0DD0400EE66E09
:1002F000B00EE66E010EE66E89EC05F0E552E552B1
:10030000E5520001636B11D06D926D6ADF6AFF0EDA
:10031000DF5C09E2E868E85004E0E80600D000D0BD
:10032000FAD7DF2AF4D7FF0000D0E552E552E7CF35
:10033000D9FF1200D9CFE6FFE1CFD9FF030EE126A6
:10034000010EDB6A66C000F0016A026A005000011B
:10035000675DF66E015000016859F76E02500001AA
:100360006959F86E0F0EF614E76E020EE7CFDBFF49
:10037000F00EF616DF6A100EDF5C1EE2020EDB5096
:1003800015E1000166510FE0010EDB50EA6A6B0FC8
:10039000E96E000EEA22EF50F56E0D00010EDB2A29
:1003A0000001660702D0F5680D0004D0F5680D0065
:1003B000020EDB06DF2ADFD70A00A40EA66E4CD899
:1003C000DF6A00016651DF5C15E2010EDB50DF24BD
:1003D000EA6A6B0FE96E000EEA22EF50E66EDF501C
:1003E000EA6A6B0FE96E000EEA22E552E750EF6E03
:1003F000DF2AE7D7030EE15C02E2E16AE552E16E33
:10040000E552E7CFD9FF1200D9CFE6FFE1CFD9FF00
:10041000E65271C1F6FF72C1F7FF73C1F8FFDF6AE0
:1004200001017551DF5C13E23A0E0101D880755568
:10043000DF24EA6A760FE96E010EEA22EF50F56ECC
:100440000C00C40EA66E08D80900DF2AE9D7E552D1
:10045000E552E7CFD9FF1200F29E550EA76EAA0E05
:0C046000A76EA682A6B2FED7A6941200DA
:04046C006C500CE1E3
:100470006896040100513C0BE842E8420D0802E195
:100480000AD8010C3BD8010C040E6C5C03E16896A1
:1004900044D8010C000C70D9E652040104BF046B6F
:1004A0000001B36BAB6BAC6BB16BB26BCDEC03F01B
:1004B000DF6ADF50006E016A010E005C000E015819
:1004C0001AE20001AC5117E1F76ADF34FE0BF73690
:1004D000F66EEC0EF6260D0EF7220900F5CF00F0B1
:1004E0000800F5CF01F004D001C0FAFF0050F96E0A
:1004F000FBDFDF2ADED7ACD8E55243D1020E000184
:10050000AB5D09E179D8040100BD02D0C80E01D06D
:10051000880E006F120061EF03F0040E0101FA5D16
:1005200009E112C46EFF6E50000802E2050E01D010
:10053000030EFA6F0001AB0510E111D8020E0001A5
:10054000B35D03E10401840E06D0040104BD02D0B2
:10055000C80E01D0880E046F120061EF03F00CD9B1
:10056000020EE1260001080EB15D000EB2590DE247
:10057000B1C0DEFFB2C0DDFFB35102E1010E03D016
:10058000B30506E1020EB36F03D0080EDE6EDD6A1E
:10059000040104930491010EDB500413DFCF05F432
:1005A000000EDB500001B15F010EDB50B25B180E94
:1005B000AF6F040EB06F0101FBA30CD0D6D815E0CD
:1005C000ADC0F6FFAEC0F7FF0800F550BED8F6E2AA
:1005D000DB06F4D7CAD809E0ADC0E9FFAEC0EAFF38
:1005E000EF50B3D8F7E2DB06F5D7020EE15C02E28A
:1005F000E16AE552E16EC5D0BFD8020EE126030ED6
:1006000004010015E76E010EE7CFDBFF01C4DFFF39
:10061000DE500001B127DD50B223180EAD6F040E7D
:10062000AE6FA3D80EE0ADC0E9FFAEC0EAFFEF5059
:10063000AFC0E9FFB0C0EAFFEF6EA7D8F2E2DB0679
:10064000F0D7020EE15C02E2E16AE552E16E99D078
:100650006D980001AC5105E180D8840E006F040153
:100660001DD0040110AF1CD00001B1510401165D72
:100670000001B2510401175904E216C4B1F017C4C5
:10068000B2F06DDF0001010EAB6F67D8800E006F16
:100690000401180E066F040E076FC80E046F1200D7
:1006A0000001020EAB6F0401056BC80E046F04015C
:1006B000080E016F180E026F040E036FC80E006F54
:1006C00012005AD8E652020E0001AB5D35E16D50C2
:1006D000100B32E004010151006E016A080E00188F
:1006E0002BE1015029E100513C0BE842E8420D08A2
:1006F00023E10051800B20E1100E026F040E036F06
:10070000DF6ADF50006E016A080E005C000E0158BF
:100710001AE2DF50EA6A180FE96E040EEA22EF507F
:10072000E66EDF50EA6A100FE96E040EEA22E55227
:10073000E750EF6EDF2AE5D70001AB6B0ED88C0EC9
:10074000006F0401046BE5521CD0AFC0E9FFB0C0DC
:10075000EAFFEF6E0001C5EF03F00401080E016F20
:10076000100E026F040E036F1200D9CFE9FFDACF2B
:10077000EAFFEE50ED101200D9CFE6FFE1CFD9FF2E
:100780001200E552E7CFD9FF1200AF2B000EB023C5
:0A079000AD2BAE23DF06010E1200B0
:06079A0004011051600B88
:1007A000E842E842E842E842E842000901E012007B
:1007B0001151070A40E00B0A3EE0070A33E0010A44
:1007C00023E00B0A1FE0020A1DE0030A19E0080AF1
:1007D00010E0010A0CE00F0A08E0030A01E0120031
:1007E00012D90101040EFA6F12001CEF04F053EF4E
:1007F00004F009D90001FC0EAD6F010EAE6F0CD0F4
:100800006EEF04F0A0EF04F002D90001AD6FAE6B03
:10081000FD0EAD27010EAE230101FB930001010E79
:10082000B16F1200F4D8EA6AFD0FE96E010EEA22F8
:1008300012C4EFFF12001200800E0401105D32E1BD
:100840001351030A1FE0010A0AE0030A29E1DBD879
:1008500000012C0EAD6F0D0EAE6F120E1ED0B2D871
:10086000E20EF6260D0EC0D8020E0001F76AAD2585
:10087000F66EAE51F7220900F5CFB1F00A00F5CFC0
:10088000B2F00ED09FD8E60EF6260D0EADD8ADC054
:10089000F6FFAEC0F7FF0800F5500001B16FB26B74
:1008A0000101FB831200AFD80F0EE66E710EE66EEB
:1008B0000F0EA2D8010EE66EFD0EE66E010E9CD85C
:1008C00012C4FCF10401125104E10101050EFA6F9A
:1008D00012000101060EFA6F74EF05F00401186BA7
:1008E000196B040110511F0B020A0FE0030A0BE001
:1008F000010A18E188D8040118810101FBA112D076
:10090000040118830FD07FD80DD050D801E0010E1C
:1009100062D8AFC0E9FFEA6EEF50040B03E00401B8
:10092000010E186F0001AC050AE10001180EAD6F51
:10093000040EAE6F0101FB930001020EB16F1200B5
:10094000040112050EE110511F0B00090AE15BD8EA
:10095000030E0401115D03E10101FB8102D00101DD
:10096000FB910401125121E110511F0B02081DE1FE
:1009700014510F0B000919E019D801E0010E2BD812
:10098000030E0401115D02E1840E03D014AF07D001
:10099000400EAFC0E9FFB0C0EAFFEF6E1200880E54
:1009A000AFC0E9FFB0C0EAFFEF6E120030D80F0B06
:1009B000080DF350016A000F006E040E012214515D
:1009C000800B120020D804011251F66EF76AD890FD
:1009D000F636F7361200040DF35000010024AF6F15
:1009E000000E0120B06F1200F7220900F5CFADF024
:1009F0000A00F5CFAEF01200E66E81EC06F0E5528B
:100A0000E552E55212000001010EAC6F1200FBDF4F
:060A100004011451120064
:0A0A1600040110511F0B010801E05C
:100A20001200145101E01200060E115D24E1135171
:100A3000230A1FE0010A0DE0030A1BE1DBD80101D4
:100A4000FC0505E10001500EAD6F0D0EAE6F090EF5
:100A50000DD0D0D80101FC0505E10001C50EAD6F38
:100A60000D0EAE6F0101FC0504E11D0E0001B16F1A
:100A7000B26B0101FB8304011051600BE842E842B4
:100A8000E842E842E842010801E0120011510B0A75
:100A900025E0080A17E0090A11E0080A09E00B0A34
:100AA00005E0080A01E0120072EF05F073EF05F0AF
:100AB000A1D80001B40EAD6F000E09D09BD813C4AD
:100AC000B4F0120097D80001B50EAD6F000EAE6FF6
:100AD0000101FB930001010EB16F12008BD812C40B
:100AE000B5F01200120012000001B66B1E0E716EFE
:100AF0000401400E096F200E0A6F040E0B6F880E62
:100B0000086F0401600E0E6F040E0F6F400E0C6F25
:100B10001200D9CFE6FFE1CFD9FFE652FC0EDB5041
:100B2000400805E2400EF36EFC0EF3CFDBFFDF6AF8
:100B3000FC0EDB50DF5C0FE2DF5050D8EF50E66E6A
:100B4000DF50EA6A600FE96E040EEA22E552E750D0
:100B5000EF6EDF2AEDD7FC0EDBCF0DF4400E040163
:100B60000C170C7D880E0C13E552E552E7CFD9FF28
:100B70001200D9CFE6FFE1CFD9FF0001B66B040127
:100B800008BF26D0FC0EDBCF00F00951D8800054FE
:100B900003E2FC0E09C4DBFF0001B66BFC0EDB5068
:100BA000B65D0FE2B651EA6A200FE96E040EEA2242
:100BB000EF50E66EB65112D8E552E750EF6EB62B05
:100BC000EDD70401400E096F0817087D880E081341
:100BD0000001B651E552E7CFD9FF1200E76EFD0ED6
:100BE000DBCFE9FFFE0EDBCFEAFFE750E926000E80
:0C0BF000EA2212000001020EAC6F12009D
:040BFC006DA60CD8FE
:100C00000101FA0508E16DBA06D0686A696A69806F
:100C10006988020EFA6F12006D6A696A6D860101B9
:100C2000010EFA6F12006D6A696A0101FA6B120017
:100C300013EF06F00101FA5101E1120068B425D862
:100C40006DB2120068B038D868B817D868BA24D81E
:100C5000030E0101FA5D01E212000001B76B040E00
:100C6000B75D0AE268A608D036EC02F0000901E19F
:100C700068960001B72BF3D71200698468986D82DB
:100C8000A19AA08A0300A09A12006D92699468A4A8
:100C900002D06894FCD7120070A00CD0800E040122
:100CA000005D07E1840E0401045D03E104018C0E84
:100CB000006F7090689A12006A6A686A9F0E6B6E85
:100CC0007B0E696E6E6A0F0EE66E710EE66E0F0E8B
:100CD000E66E17D8E552E552E552160E706E68A61C
:100CE00005D0689600D000D00000F9D76D9861EC6F
:100CF00003F00101FB910101FC6B0101030EFA6F8E
:100D00001200D9CFE6FFE1CFD9FFFD0EDBCFE9FF1F
:100D1000FE0EDBCFEAFFFC0EDB5004E0EE6AFC0EB9
:0C0D2000DB06F9D7E552E7CFD9FF12003F
:040D2C0012010002AE
:100D300000000008D8043C00020001020001090282
:100D40002900010100C03209040000020300000074
:100D5000092111010001221D000705810340000146
:100D6000070501034000010403090434034D006931
:100D700000630072006F006300680069007000206B
:100D80000054006500630068006E006F006C006F27
:100D90000067007900200049006E0063002E0026E5
:100DA0000348004900440020005500530042002041
:100DB0000042006F006F0074006C006F00610064FF
:100DC00000650072000600FF0901A1011901294018
:100DD000150026FF007508954081021901294091F0
:0E0DE00002C03E0D3E0D670D6B0D9F0D160AF5
:020DEE00200ED5
:100DF000F66E000EF76E000EF86E01010900F55058
:100E0000F56F0900F550F66F03E1F56701D03DD0AD
:100E10000900F550F06F0900F550F16F0900F55029
:100E2000F26F09000900F550E96E0900F550EA6E0D
:100E3000090009000900F550F36F0900F550F46F3F
:100E400009000900F6CFF7F1F7CFF8F1F8CFF9F183
:100E5000F0C1F6FFF1C1F7FFF2C1F8FF0101F35352
:100E600002E1F45307E00900F550EE6EF307F8E2F3
:100E7000F407F9D7F7C1F6FFF8C1F7FFF9C1F8FF9A
:0C0E80000101F507000EF65BBFD7120061
:040E8C000F0EC16E16
:100E900081A804D0070EC16E00EF08F00ED8040040
:100EA00016D819D8060E0101FA5D05E16D50020B46
:100EB00002E123EC00F0F3D71200140E6F6E010173
:100EC000FA6B0101FB6B0101FC6B17EF00F0FEEC0C
:100ED00005F01AEF06F00101FE51FF1104E1100EBA
:100EE000FE6F270EFF6FFE07000EFF5B060E01016F
:100EF000FA5D02E28C8008D00101FE51FF1107E18A
:100F00008C708C50010B02E08C9212008C821200CB
:100F100011EE00F021EE00F0F86A049CF7EC06F008
:0C0F20009DEC07F046EC07F0FBD7120038
:040F2C0000EE00F0E3
:0A0F30000F0EEE6AEA62FDD7120010
:020F3A001200A3
:020F3C000000B3
:020000040030CA
:0100000024DB
:010001000EF0
:010002003FBE
:010003001EDE
:01000500807A
:010006008178
:0100080003F4
:0100090040B6
:01000A0003F2
:01000B006094
:01000C0003F0
:01000D0040B2
:00000001FF
